:1000000010C01FC01EC01DC01CC01BC01BC019C01B
:1000100018C017C016C015C014C013C012C011C03C
:1000200010C011241FBECFE5D1E0DEBFCDBF10E070
:10003000A0E6B0E001C01D92A536B107E1F7E7D018
:100040006DC1DECF1F920F920FB60F9211248F93C6
:100050009F931DBC1CBC9091610080916200981719
:1000600041F08091610080936300809161008093F2
:10007000620080916100882329F0809163008F5F86
:100080008093630080916300893921F0809163003F
:100090008A3009F4C19A80916300833121F4C198B8
:1000A00081E08093630080916300853A21F4C198D8
:1000B00086E98093630081E0809364009F918F9133
:1000C0000F900FBE0F901F901895882319F0813064
:1000D00031F403C0C29AC0980895C298C09A089596
:1000E000882321F410926100C1980895813029F489
:1000F0001DBC1CBC809361000895823021F41092D5
:100100006100C19A0895833029F41DBC1CBC86E9A6
:1001100080936100089540E027E030E051E061E025
:1001200070E0DC98852F8A95F1F7CD9B08C0CB0154
:10013000022E02C0880F991F0A94E2F7482BDC9A1E
:10014000852F8A95F1F7215030408FEF2F3F3807E8
:1001500041F7842F0895DF93CF930F92CDB7DEB789
:10016000898347E050E0FE01319661E070E0A1E054
:1001700080819B01042E02C0220F331F0A94E2F7F4
:1001800090E0282339231216130614F4DE9A01C0D6
:10019000DE98DC988A2F8A95F1F7DC9A8A2F8A9567
:1001A000F1F7415050408FEF4F3F580709F7DE9A63
:1001B0000F90CF91DF9108950F931F93182F062F63
:1001C000DF9880E2C8DF812FC6DF802FC4DFDF9A8F
:1001D0001F910F9108951F93182FDF9880E2BBDFC6
:1001E000812FB9DFDF9A82E08A95F1F7DF9881E20B
:1001F000B2DF91DFDF9A1F9108958F5F682F660F3E
:10020000660F660F8068682B84E0D6DF08951F9321
:10021000CF93DF9387B3876087BBD198D99AD29A5F
:10022000D39AD79A8AB380658ABBD598619A88EBAE
:100230009BE09BBD8ABD8EB584608EBDDF9ADA9847
:10024000DB98C29AC09AC19A80E29EE428EC30E022
:10025000F9013197F1F70197D9F7DA9ADB9A81E042
:1002600034DF80E068E0A8DF81E064E0A5DF82E0C1
:100270006BE0A2DF83E065EC9FDF81E0BEDF85E01D
:1002800060EE9ADF86E06FE797DF789411E0C8ECC4
:10029000D0E0C9991FC084EF91E0FE013197F1F7DA
:1002A0000197D9F784EF91E0FE013197F1F70197BB
:1002B000D9F7C99B0FC084EF91E0FE013197F1F7A8
:1002C0000197D9F784EF91E0FE013197F1F701979B
:1002D000D9F719C0809164008130D9F68CE07BDFBA
:1002E000867011F081E00BC08BE075DF86FF06C0E1
:1002F00081FF02C083E003C082E001C080E0F0DE45
:1003000010926400C6CF812F8F5F10E0823009F019
:1003100011E0812FDADE812F70DFDCCFF894FFCF80
:00000001FF
